:100000000C94A2010C94E9010C94E9010C94260DC6
:100010000C94E9010C94E9010C94E9010C94E901B8
:100020000C94E9010C94E9010C94A61E0C947A1F1F
:100030000C9466190C94E9010C94E9010C94E90103
:100040000C94E9010C94E9010C94E9010C94E90188
:100050000C94E9010C94BD190C94E9010C94E9018C
:100060000C94E9010C94E9010C94E9010C94E90168
:100070000C94E9010C94E9010C94E9010C94E90158
:100080000C94E9010C94E9010C94E9010C94E90148
:100090000C94E9010C94E9010C94E9010C94E90138
:1000A0000C94E9010C94E9010C94E9012900140075
:1000B0001A000800150017002B000400166A0764D8
:1000C00009680A6101001D001B00060019000500F7
:1000D00000000000E10091622C422A002D00130074
:1000E00012000C0018001C00290033000F6A0E6477
:1000F0000D780B7101003800370036001000110038
:1001000000000000E500906228412A000100310053
:100110001E022402310200000100200235003402D8
:10012000340035020100010001002F022F002602D9
:1001300000000000010001002A0001002D00220241
:1001400025022E022E000000010021024F00520065
:1001500051005000010023021F023002300027022C
:1001600000000000005C010001000100010001002E
:10017000010001000100000001001E001F0020001E
:100180002100220001000100010001000100010026
:1001900000000000005C0100010001002D002202AF
:1001A00025022E022E000000010027002600250057
:1001B0002400230001003800370036000100010050
:1001C00000000000010001004C00010000000000E0
:1001D000000000002A2B28000000000000000000A2
:1001E0000000000000000029000000002C1E342048
:1001F000212224342627252E362D3738271E1F206E
:100200002122232425263333362E37381F040506B2
:100210000708090A0B0C0D0E0F10111213141516F6
:100220001718191A1B1C1D2F3130232D35040506F4
:100230000708090A0B0C0D0E0F10111213141516D6
:100240001718191A1B1C1D2F3130354C00000000E7
:10025000000000000000000000000000000000009E
:100260007E0F00D4FFFFFFC7000000780E0363007D
:100270006C00610077003400340000000C0379004A
:10028000660075006B007500000004030904090294
:100290004200020100A0FA0904000001030101006C
:1002A0000921110100012240000705810308000A0D
:1002B00009040100020300000009211101000122CC
:1002C0002200070582032000010705030320000127
:1002D000120110010000000846590100010001024E
:1002E00000010660FF0961A1010962150026FF00F7
:1002F0009520750881020963150026FF0095207579
:10030000089102C005010906A101050719E029E7C6
:100310001500250195087501810295017508810177
:100320000507190029FF150026FF009506750881AD
:1003300000050819012905950575019102950175BA
:10034000039101C011241FBECFEFDAE0DEBFCDBFA5
:1003500004B603FE27C08091E0019091E101A091D5
:10036000E201B091E3018730904BA740B04BD1F44C
:100370001092E0011092E1011092E2011092E3016B
:1003800014BE84B7877F84BF0FB6F894A895809178
:100390006000886180936000109260000FBEE0E012
:1003A000F8E3099511E0A0E0B1E0E8E6F3E402C06B
:1003B00005900D92A432B107D9F721E0A4E2B1E093
:1003C00001C01D92A03EB207E1F70E94621B0C948F
:1003D0007B210C9400008E3024E6920771F030F4FB
:1003E0008730944651F084EB90E008958F302AE6F0
:1003F000920719F086319A46B1F786EE90E008959B
:100400000895CF93FB01C2818A32FDE59F0781F0F9
:100410008B322DE5920791F089329D45A1F4CC23D2
:1004200021F080E00E942A03C0E08C2FCF91089534
:1004300082E0CC2329F00E94DF15F6CF81E0F9CFCE
:100440000E940016F2CFC1E0F0CF81E008950C9435
:10045000010208950C9429021F93CF93DF9300D0DB
:1004600000D00F92CDB7DEB749835A836B833091AA
:10047000430189819A8131111DC06623B9F022237D
:10048000A9F00E94D216182F682F89819A810E94A4
:100490007B1669817A81812F0F900F900F900F90BA
:1004A0000F90DF91CF911F910C9481090E94A916A2
:1004B000182FEFCF0E94D21669817A81EDCFFC010F
:1004C000262F408151816281738184810C942C029A
:1004D000CF93DF93EC0160E00E945F02BE01DF91E9
:1004E000CF910C942A02FF920F931F93CF93DF9327
:1004F000E82FF0E0E453FE4FF490C82FC695C69560
:10050000C695D0E0FE01E45AFD4F0491877010E0DB
:10051000082E02C0159507950A94E2F7017011277D
:10052000C45BDD4FFE01C491D0E002C0D595C795F4
:100530008A95E2F7C170DD270115110519F081EEEA
:100540000E94F70E209719F086EE0E94F70E8F2D6D
:100550000E944A0FCD2B19F086EE0E94220F012B2C
:1005600041F081EEDF91CF911F910F91FF900C949C
:10057000220FDF91CF911F910F91FF900895EF927D
:10058000FF920F931F93CF93DF93EC01162F0AE096
:100590008881882309F454C0813009F04EC08981D4
:1005A000813099F47E0122E0E20EF11C8A810E94E2
:1005B0004A0FE7012196812F815050F3EFE9FFE0C8
:1005C0003197F1F700C00000F7CF823041F47E018F
:1005D00082E0E80EF11C8A810E94F70EEACF833098
:1005E00041F47E01E2E0EE0EF11C8A810E94220FAE
:1005F000E0CF843011F02196DDCF2A81229690E061
:1006000080E0AE014F5F5F4F2053330B2A3031053E
:1006100048F0019778F2EFE9FFE03197F1F700C079
:100620000000F7CF089FB001099F700D1124C90188
:10063000860F971F2981EA01E4CF0E947302BACF87
:10064000DF91CF911F910F91FF90EF90089560E09F
:100650000C94BF02CF93DF93C1E0D0E002C0CC0F77
:10066000DD1F8A95E2F78C2F0E942218BE0190E0D0
:1006700080E0DF91CF910C947D158F929F92AF9285
:10068000BF92CF92DF92EF92FF920F931F936B0175
:100690007C0181E090E0A0E0B0E04C015D0104C08D
:1006A000880C991CAA1CBB1C4A95D2F7B501A40161
:1006B0004C015D0104C0880C991CAA1CBB1C2A9526
:1006C000D2F7482959296A297B2904C0880F991F24
:1006D000AA1FBB1F0A95D2F78A019B010C211D217D
:1006E0002E213F21041715072607370789F48C2987
:1006F0009D29AE29BF29BC01CD011F910F91FF900B
:10070000EF90DF90CF90BF90AF909F908F90089523
:1007100080959095A095B0958C219D21AE21BF210B
:10072000EACF0F93382F262F60919A0170919B0189
:1007300080919C0190919D01042F432F0E943D03C5
:100740000F910C94B9150E94F4190E940F18811191
:1007500002C00E94B8180C94BD050C94C005089501
:100760000E9492110E94AF032FEF84E39CE021507E
:1007700080409040E1F700C000000C94E1190F9315
:100780001F93CF93DF93EC0161E00E945F028C0125
:10079000BE010E94B807882359F1BE01C8010E941A
:1007A0002702882329F1BE01C8010E94D70A8823A5
:1007B000F9F0BE01C8010E94290B8823C9F0BE01CF
:1007C000C8010E944C0C882399F08A81882339F053
:1007D00001158CE5180751F00F3D1C4579F0CE014D
:1007E000DF91CF911F910F910C9425020E94B003CD
:1007F00080E0DF91CF911F910F9108950E94B8186A
:10080000F7CF08950C94010481E008950C9404043A
:10081000CF93C82F0E9402048C2FCF910C94060412
:10082000CF93DF930E9481090E94E304EC018115BC
:1008300023E5920790F5811532E5930708F096C0FD
:1008400081159042C8F4C11581E0D80788F4C53AF3
:10085000D10548F4C430D10558F4C130D10541F078
:10086000D0E0C0E005C0CE01805E91090897C0F7D6
:10087000CE01DF91CF910895C11591E5D90708F018
:1008800070C0C11520E5D20708F04EC0C11530E494
:10089000D30730F3DF70D06AEBCF811546E59407BC
:1008A000F0F4C11585E5D80708F075C0C11594E5C9
:1008B000D90708F06BC0CE018370992721E030E0A2
:1008C00002C0220F331F8A95E2F7C695C69590E2C3
:1008D000C99FE0011124C22BD32BDA68C9CF81153F
:1008E0002AE5920778F4811539E5930708F05EC090
:1008F000811548E5940708F4B3CFD82FCC27C06FF3
:10090000D06AB6CF90568115904208F0A9CF8D2FAE
:100910008F710E947A0590E0982F882788279F7111
:100920009C012C2BE90140C0CE01E4E0969587950F
:10093000EA95E1F783702C2F26952695237040E2E7
:10094000249F90011124382B8C2F8370C1E0D0E0BC
:1009500002C0CC0FDD1F8A95E2F7C22BD32BDC68D7
:1009600087CFDC2FCC27C16FD06A82CF83709927C5
:1009700021E030E002C0220F331F8A95E2F7C695CE
:10098000C69580E2C89FE0011124E7CFDC2FCC2779
:10099000C46FD06A6DCF8C2F0E947A05C82FD0E02B
:1009A000DC2FCC27CC27DF71D06262CF8F700E9402
:1009B0007A0534E0D695C7953A95E1F7CF709C2F2C
:1009C000EC01D06955CF82389105B1F1B0F4813393
:1009D000910509F475C048F48932910509F469C09C
:1009E0008A32910509F473C008958533910509F49D
:1009F00059C08933910501F10895833E9105A9F10C
:100A000038F4803E9105F9F0823E910549F1089550
:100A1000863E9105A9F1873E9105C9F1843E910575
:100A200019F52091D20121FF1FC08091D10184FDD1
:100A300014C087EE90E008952091D1012370A1F0B9
:100A400080EE90E008952091D10120FD47C03091C3
:100A5000D20130FF09C024FF44C090E080E004C010
:100A60002091D10122FDF7CF08952091D10122FDDF
:100A70003BC03091D20130FDE3CF24FFF5CFEDCF65
:100A80002091D10123FFF0CF24FDE7CFD2CF2091D9
:100A9000D10123FD2CC03091D20131FFEECF84EE85
:100AA00090E008952091D10125FFDECF89E290E00A
:100AB00008952091D10125FFD7CF85E390E00895D7
:100AC0002091D10126FFD0CF8AE290E008952091B5
:100AD000D10126FFC9CF81E390E0089589E390E03A
:100AE000089583EE90E0089582EE90E0089586EEFA
:100AF00090E008959091D10192FF06C0282F2871AF
:100B00002830F9F4877F846093FF06C0282F28716E
:100B10002831F1F4877E84612091D20120FF06C044
:100B2000382F38713830D9F4877F816021FF06C0B3
:100B3000282F28712831D1F4877E816194FD877E2A
:100B40000895282F24712430F9F68B7F8860DCCF3C
:100B5000282F2471243101F78B7E8861DDCF382F57
:100B60003171313019F78E7F8860E0CF282F2171E5
:100B7000213121F78E7E8861E1CF0C940002089527
:100B80000C94BF05E82FF0E0ED53FE4F80810895EF
:100B9000089580EA8A95F1F70895F894E82FE29590
:100BA000EF70F0E031A1282F2F7081E090E001C0BC
:100BB000880F2A95EAF7982F9095932391A392A1F5
:100BC000892B82A37894089508950E941C07809130
:100BD00000018091000194E0811190E09093CC019C
:100BE00084E0891B8093CB0184E90E94CD0586E6D1
:100BF0000E94CD0587E90E94CD0586EC0E94CD05B7
:100C000084EF0E94CD0585EF0E94CD0586EF0E94FE
:100C1000CD0587EF0E94CD0581E30E94CD0583E3DA
:100C20000E94CD05EBEBF1E0A3ECB1E083EC91E0A9
:100C300011921D928E179F07D9F784E00E94C70674
:100C40000E94A3030C9426070E94FE068823F1F05D
:100C50008091CB0190E08D539E4F0E943907811106
:100C600012C0809124018F5F80932401863048F068
:100C7000E091CB01F0E0ED53FE4F10821182128221
:100C800013820C94AD0310922401FBCF8091CC0110
:100C900090E08D539E4F0E9452070C94E405CF9232
:100CA000DF92EF92FF920F931F93CF93DF93CCE1EC
:100CB000D1E00BEB11E0D12CEE24E394F12C8991DF
:100CC000F894E82FE295EF70F0E021A18F70A70172
:100CD00002C0440F551F8A95E2F7CA01922F982B44
:100CE00091A392A18095892382A378940E94C9053B
:100CF000E6E1F1E030E020E0C12C4191A42FA29583
:100D0000AF70B0E090968C9190E04F7002C09595D6
:100D100087954A95E2F780FD36C08E2D022E01C0E0
:100D2000880F0A94EAF7C82A2F5F3F4F2630310513
:100D300021F7FE01319780810E94CD05F801808165
:100D4000C81619F1C08281E0D82A0F5F1F4FF1E069
:100D5000C032DF0709F0B3CF6091CC0170E06D5372
:100D60007E4F2D2D44E08BEB91E00E94C8060E943F
:100D700024068D2DDF91CF911F910F91FF90EF9061
:100D8000DF90CF90089580E0CECF80E0DDCF089552
:100D9000FF920F931F93CF93DF93F82E092F162FF7
:100DA000D72FC42F222349F081E0809327010E948E
:100DB000961990932601809325018091270188231D
:100DC000A1F080912501909126010E94AE1906970D
:100DD00060F0EF2DF02FA12FBD2FCE0FDF2FD11DF3
:100DE000EC17FD0741F410922701DF91CF911F917D
:100DF0000F91FF90089581918D93F2CF80912801FA
:100E0000811111C08091D80080618093D8008AE15F
:100E10008A95F1F700C09091D900892F817090FFD9
:100E200082E08093280181E090912801913009F0BF
:100E300080E008950C94FE060E941A07809300013A
:100E40000E94FE0681110C942D0708950E94FE0653
:100E5000811102C00C943307089561E070E081E0D5
:100E600091E00C94D70C61E070E081E091E00C948B
:100E7000DE0CCF93DF93D82FC92F0E94780D0097F7
:100E800079F4ED2FFC2FDC01A65DBE4F2C91219350
:100E9000019684309105B9F781E0DF91CF910895F3
:100EA00080E0FBCF30E020E0FC014191CF01F9016F
:100EB000E65DFE4F40832F5F3F4F24303105A1F7A1
:100EC000089582E290E00E943921813289F483E220
:100ED00090E00E943921823059F484E290E00E942F
:100EE000392191E0823109F090E0892F81700895D5
:100EF00080E0FCCFCF93C82F6FEF811161E282E2D7
:100F000090E00E9447216FEFC11162E083E290E020
:100F10000E9447216FEFC11162E184E290E0CF911E
:100F20000C94472180E00E947A070C9409180895D8
:100F300085E290E00E943921682F70E090E080E027
:100F4000089585E290E00C9447210E9497070E9443
:100F5000610781110CC060E070E0CB010E94A10725
:100F60000E94F9080E94E50981E00C947A0708952F
:100F7000CF93FB01C281CC2309F19C0122513F4553
:100F80002031310520F582510E94F509C0E08C2FF7
:100F9000CF91089581E00E94DF1543E062E081E097
:100FA0000E949103F3CF81E00E94001643E062E0CB
:100FB00081E00E949103EBCF82E0F6CF8031FFE524
:100FC0009F0789F381319F45B9F3C1E0E0CF8031BC
:100FD000EFE59E07F9F281319F45C9F682E0DBCF4C
:100FE0002FEFFC0120830895EF92FF920F931F9340
:100FF000CF93DF93EC01062FE881E150E33108F055
:101000005EC0F0E0E358FE4D0C942C21198289E07B
:101010008A83602FCE01DF91CF911F910F91FF90B6
:10102000EF900C945D1A8981823069F0833071F001
:101030008130D9F40E94A2190E9432216A837B83F5
:101040008C839D83E6CF0E949807F6CF7E0122E035
:10105000E20EF11C10E0812F0E94C205F70181937E
:101060007F011F5F1830B9F7D4CF602FCE010E94E7
:10107000F007CFCF89818230C1F76A817B818C8173
:101080009D810E9432210E94A107C3CF4B816A81BA
:1010900089810E94CB089827892798279D838C8374
:1010A000B8CF2C813D813227232732274B816A819B
:1010B00089810E94E408ADCF0E94F908AACF8FEF82
:1010C0008883A7CF0E948E098983A3CF0E949009AD
:1010D0009827892798279A8389839BCF6B8170E013
:1010E00089819A81AE014C5F5F4F982789279827A5
:1010F0000E9493098ECF6B8170E089819A81AE0145
:101100004C5F5F4F9827892798270E94BA0981CFA3
:101110000E94E5097ECF0E94B908D6CF6B8170E0AE
:1011200089819A81AE014C5F5F4F98278927982764
:101130000E9431096ECF6B8170E089819A81AE0186
:101140004C5F5F4F9827892798270E94570961CFE6
:101150000E9492075ECF0E945D1AFFEF21EE84E0AD
:10116000F15020408040E1F700C000000E94E119EA
:1011700050CF84E0089550E0440F551F9CE0699FD4
:10118000400D511D112490E6899F400D511D1124E1
:10119000CA01869608950F931F93CF93DF930E9401
:1011A000BB088C010E943921C82FD0E0DC2FCC274E
:1011B000C80101960E9439219E01282BC901DF91A7
:1011C000CF911F910F9108950F931F93CF93DF93AA
:1011D000122F032F0E94BB08EC01602F0E944721B1
:1011E000612FCE010196DF91CF911F910F910C9449
:1011F0004721AF92BF92CF92DF92EF92FF921F935F
:10120000CF93DF938CEAC82E80E0D82ED0E0760111
:10121000C0E014C0F50125913491412F6C2F8D2F22
:101220000E94E40882E0A80EB11C1F5F163091F7FF
:101230008CE0E80EF11CCF5FC83019F0570110E0C8
:10124000E9CFDF5F80E6C80ED11CD43001F7DF9113
:10125000CF911F91FF90EF90DF90CF90BF90AF9014
:101260000895EF92FF920F931F93CF93DF93EC01BA
:101270008A017C01E60EF71ECE018696CE15DF05AB
:1012800039F4DF91CF911F910F91FF90EF90089566
:10129000C03821E0D20740F40E943921F801808350
:1012A0000F5F1F4F2196E8CFF8011082F9CFCF9240
:1012B000DF92EF92FF920F931F93CF93DF937C0106
:1012C0006A018C01060F171FEC01CE018696C0172C
:1012D000D10749F4DF91CF911F910F91FF90EF90CB
:1012E000DF90CF900895C03821E0D20740F4FE018E
:1012F000EE19FF09EC0DFD1D60810E94472121962A
:10130000E4CF462F843038F4783028F4663018F46F
:10131000672F0C94CB0890E080E0089580E1089559
:101320008AE592E00895EF92FF920F931F93CF9377
:10133000DF93EC018A017C01E60EF71ECE018A558F
:101340009E4FCE15DF0539F4DF91CF911F910F919C
:10135000FF90EF900895CA3522E0D20740F40E9432
:101360003921F80180830F5F1F4F2196E7CFF801E5
:101370001082F9CFCF92DF92EF92FF920F931F93DB
:10138000CF93DF937C016A018C01060F171FEC01DC
:10139000CE018A559E4FC017D10749F4DF91CF91F6
:1013A0001F910F91FF90EF90DF90CF900895CA3575
:1013B00022E0D20740F4FE01EE19FF09EC0DFD1DFD
:1013C00060810E9447212196E3CFCF93DF93C6EA45
:1013D000D1E060E0CE010E9447212196C11584E052
:1013E000D807B9F7DF91CF910895DF92EF92FF927E
:1013F0000F931F93CF93DF9300D000D0CDB7DEB70C
:10140000F82E8FE08F1540F08FEF93E00E94392186
:1014100006EA11E08823C1F00F900F900F900F9013
:10142000DF91CF911F910F91FF90EF90DF90089582
:10143000011584E0180781F3C8010E943921811148
:1014400001C0FA940F5F1F4FF110F2CF19821A8278
:101450001B821C82DD24D39478018FEFE81AF80AEE
:10146000C8010E94392189831A828823A9F29FEF3B
:10147000980F933078F48A83D9820E5F1F4FC7018B
:101480000E9439218B83882339F2CE0101960E9474
:101490002703E2CF8701F9CFAF92BF92CF92DF92BD
:1014A000EF92FF920F931F93CF93DF937C015B0129
:1014B000C42FD22FFC0182818823F9F040933001A0
:1014C0000E94961990932F0180932E0180E28C0F39
:1014D000883008F061C0C77081E001C0880FCA95EC
:1014E000EAF7DF91CF911F910F91FF90EF90DF907E
:1014F000CF90BF90AF900C945D0F109130011413FA
:1015000040C080912E0190912F010E94AE196C0174
:10151000B701C5010E94EB01C816D90690F5C0E2DB
:10152000CD0F1D17B9F080E2810F883040F417709D
:1015300081E001C0880F1A95EAF70E94640FC83055
:1015400048F481E09D2F977001C0880F9A95EAF7C3
:101550000E945D0F802F0E944A0FC830E8F4D770B8
:1015600081E001C0880FDA95EAF7DF91CF911F91F2
:101570000F91FF90EF90DF90CF90BF90AF900C94C1
:10158000640F80E28C0F883038F4C77081E001C0AE
:10159000880FCA95EAF7E9CFDF91CF911F910F919C
:1015A000FF90EF90DF90CF90BF90AF9008950F9392
:1015B0009C01CB01243F4CE5340759F1A8F4293DA7
:1015C000FCE53F0701F12A3D4CE53407D1F1283D08
:1015D0003C4591F406E221EE41EE68ED7CE50E9487
:1015E0004C0A80E00F910895263FFCE53F07E9F0A3
:1015F000B0F0273F3C45F9F0FC018281882339F1A6
:1016000010923001EFCF07E225EE45EE69ED7CE563
:10161000E6CF06E221EE40EE64EF7CE5E0CF07E2A4
:1016200025EE44EE65EF7CE5DACF06E221EE42EEF0
:1016300066EF7CE5D4CF07E225EE46EE67EF7CE56A
:10164000CECF08E221E045EE6AED7CE5C8CF81E02F
:10165000C9CFCF93DF93EC01FB018281882309F48A
:1016600019C1C230FCE5DF07C0F1C6319CE5D907DE
:1016700030F09E012B5F3C452930310570F50E940A
:1016800027189093D2018093D101C031ECE5DE0799
:1016900009F4CFC008F05BC0C8308CE5D80709F466
:1016A000B6C088F5C430ECE5DE0709F4A8C0C0F484
:1016B000C2308CE5D80709F49CC08091D1018260CA
:1016C000C330DC4509F498C08091D1019091D201DA
:1016D0000E9435180E94921180E0DF91CF91089509
:1016E0008091D1018061C630ECE5DE0709F484C049
:1016F0008091D1018860C730DC4508F47DC08091BD
:10170000D101806279C0CC308CE5D80709F489C05A
:1017100070F48091D1018C60CA30ECE5DE0709F4E9
:101720006BC008F478C08091D1018E7F65C0CE3047
:101730008CE5D80709F479C08091D1018B7FCF3037
:10174000DC4508F459C08091D1018F7E55C0CC3F53
:10175000ECE5DE0709F457C030F5C3318CE5D80756
:1017600009F46FC078F4C131ECE5DE0709F465C017
:10177000C231DC4509F0A8CF0E9492118091D101BD
:101780008F773AC0C5318CE5D80709F462C008F4F8
:1017900076C08091D2018160CB3FDC4509F094CFC7
:1017A0008093D20191CFC115FDE5DF0709F44DC04B
:1017B00088F48091D2018D7FCE3F9CE5D90781F3DB
:1017C0008091D2018E7FCF3FDC4550F38091D201D2
:1017D0008360E6CFC230FDE5DF0709F459C008F4A5
:1017E00044C080E0C330DD4509F06ECF0E94BA18D6
:1017F0006BCF8091D10181608093D10165CF8091C1
:10180000D1018460F9CF8091D2018260C9CF8091EB
:10181000D1018064F1CF0E9492118091D101806842
:10182000EBCF8091D1018D7FE7CF8091D101877F70
:10183000E3CF8091D1018F7DDFCF8091D1018F7B6C
:10184000DBCF8091D101837FD7CF8091D2018C7F74
:10185000A7CF8091D10182FB992790F921E09227AF
:1018600090FB82F990FB83F9C7CF8091D201982F2A
:10187000909591708E7F892B90FB81F991CF0E947A
:1018800092119091D101892F97FB87F98058B4CF9D
:1018900081E0ACCF81E021CFCF93DF93EB018631A4
:1018A0009C4511F50E9467179A81992399F08A7ACD
:1018B00091E009F490E090933101811109C089E22F
:1018C0000E9442170E94A61780E0DF91CF910895F1
:1018D00085E3F6CF80913101811104C089E20E9435
:1018E0004917F0CF85E3FBCF81E0EFCF8EE14A9B34
:1018F00002C08150E1F74A9BFECF08955A9880E2DA
:101900008A95F1F75A9A0895FC013BE03A95F1F770
:1019100098E020E080E031E040E14A95F1F7880F5F
:101920004A9B02C08160232742E04A95F1F70000FC
:1019300040E14A95F1F7915079F790E19A95F1F7E6
:1019400099B132E03A95F1F7000040E14A95F1F79C
:1019500092FB992790F992272081920F9083089506
:10196000EF92FF920F931F93CF93DF930F92CDB718
:10197000DEB719828C017C01E60EF11C0E151F05E5
:1019800061F481E09981911180E00F90DF91CF9116
:101990001F910F91FF90EF9008950E94760CCE0159
:1019A00001960E94840CF80181938F01E7CF9093F8
:1019B000330180933201529A5A9A089590933301D9
:1019C0008093320152985A9AEA9AE9E6F0E08081CF
:1019D0008F7C808308956150770B91E001C0990F4F
:1019E0006A95EAF720E031E0911108C0222391F0D6
:1019F0005A9A80E28A95F1F75A980895492F482318
:101A000039F05A9A232740E24A95F1F79695ECCFA0
:101A10005A98F9CF5A98EDCFFF920F931F93CF9317
:101A2000DF93EC018C01060F111DC017D10731F4B3
:101A3000DF91CF911F910F91FF900895F9900E942F
:101A40007E0C68E08F2D0E94EB0CEFCF1F920F925F
:101A50000FB60F9211242F933F934F935F936F9381
:101A60007F938F939F93AF93BF93CF93DF93EF9326
:101A7000FF935A98529AC0913201D09133016D81EF
:101A8000662321F08E819F810E940C0D0E947E0CA6
:101A900080E18A95F1F75A9852985A9A80E18A958E
:101AA000F1F76A81662309F18B819C810E94B00C59
:101AB000E881F981882311F088E001C082E0808309
:101AC0000E94760CFF91EF91DF91CF91BF91AF9182
:101AD0009F918F917F916F915F914F913F912F9146
:101AE0000F900FBE0F901F901895E881F981E4CFF9
:101AF000CF93DF93C0913201D0913301F894529A81
:101B00005A9885E08A95F1F7000052985A9A80E237
:101B10008A95F1F74A9B0CC0529A5A9AE881F9814A
:101B200081E08083789481E090E0DF91CF91089507
:101B30006D81662381F08E819F810E94B00C81119E
:101B40000AC0529A5A9AE881F98182E08083789497
:101B500082E090E0EACF0E94760C80E28A95F1F76D
:101B60005A98529A80E18A95F1F76A81662321F0AA
:101B70008B819C810E940C0D0E947E0CE881F98172
:101B80001082789490E080E0D0CF909339018093D8
:101B900038010895E0913801F0913901309721F032
:101BA0000190F081E02D099480E00895E0913801E2
:101BB000F0913901309721F00280F381E02D0994F2
:101BC000089520913601309137012817390771F0B7
:101BD0009093370180933601E0913801F0913901FB
:101BE000309721F00680F781E02D09940895209127
:101BF0003401309135012817390771F09093350180
:101C000080933401E0913801F0913901309721F04F
:101C10000084F185E02D0994089585B7806885BF1B
:101C200085B7806885BF0895089508950C94140EB3
:101C300008950C94180E0E940D0E0E94150E0C941F
:101C4000160E0C94FE06089508950E948D190E94A8
:101C5000E5050E94A5070E94081A0C94190EBF9270
:101C6000CF92DF92EF92FF920F931F93CF93DF9368
:101C7000CDB7DEB72A970FB6F894DEBF0FBECDBF43
:101C80000E94230E0E94240E0E944F060E94210EE5
:101C9000882309F45CC08BE3C82E81E0D82E10E0C5
:101CA00000E0B02E802F0E94C205E82EF601F190D0
:101CB0006F01F81609F445C08091AF0181FD0E94C3
:101CC000C8059F2D9E2580E0FF24F394292F2F2106
:101CD000A1F18E83BF82EF2081E009F480E0888744
:101CE0000E9496198160782F9A8789874E815F813B
:101CF00068858A850E94C80EF801E55CFE4F8081E8
:101D0000F826F0820E94CA0D90913A01891781F15C
:101D10000E94CA0D80933A012A960FB6F894DEBF4E
:101D20000FBECDBFDF91CF911F910F91FF90EF902C
:101D3000DF90CF90BF900C9408048F5FFF0C86302B
:101D400029F60F5F1F4F0830110509F0AACF8FEF5A
:101D500089838A831B820E9496198160782F9D83D4
:101D60008C8349815A816B818D810E94C80ECACFB4
:101D70002A960FB6F894DEBF0FBECDBFDF91CF918C
:101D80001F910F91FF90EF90DF90CF90BF9008953B
:101D9000CF93DF93CDB7DEB72B970FB6F894DEBFA6
:101DA0000FBECDBF4F83588769877A878B871E8286
:101DB0001D8285E0FE013796DE01119601900D929D
:101DC0008A95E1F749815A816B817C818D819E8161
:101DD0002B960FB6F894DEBF0FBECDBFDF91CF912B
:101DE0000C94D314FC01808191810C941417CF932F
:101DF000C82F882329F18CEF8C0F813AA0F46C2F27
:101E00008091090190910A010E94D118882329F03C
:101E10008C2F0E9449170E94A6178C2F0E944217F0
:101E2000CF910C94A61780E28C0F883048F4C770CD
:101E300081E001C0880FCA95EAF70E946A17F0CFC7
:101E4000CF910895882329F19CEF980F913A20F4BF
:101E50000E9449170C94A61790E2980F983050F4FE
:101E6000877091E001C0990F8A95EAF7892F0E9447
:101E70007017F0CF9BE5980F933020F490E080E04E
:101E80000C94E10D885A873120F490E080E00C94A6
:101E9000F70D0895CF93C82F0E94F70EC93349F468
:101EA0002FEF87EE93E0215080409040E1F700C093
:101EB00000008C2FCF910C94220F882321F00E94D8
:101EC0006A170C94A6170895882321F00E947017B2
:101ED0000C94A6170895BF92CF92DF92EF92FF92D3
:101EE0000F931F93CF93DF937C01D62FC72FFC0155
:101EF000158112951F70028101110E9487170E949F
:101F00006017D82E882391F00023E9F08C2F807F72
:101F1000803421F080E28D0F8830A8F082E00E94AA
:101F2000F1170E94601791E0D82ED926CC2EC294CA
:101F30009FE0C922FBE0FC15A8F1EC2DF0E0E05792
:101F4000FE4D0C942C21D12CF1CF1C2F1F70C07F83
:101F500011F01295107F0023A9F0112359F080E2AF
:101F60008D0F883010F0D11109C0812F0E946A179F
:101F70000E94A6178D2F0E94F70E14C0812F0E9479
:101F80007A17F6CF8D2F0E94220F112359F080E28D
:101F90008D0F883010F0D1112BC0812F0E94701747
:101FA0000E94A617EC2DE850FF0B349720F40E94F6
:101FB000CA0D0E940804DD2009F461C10E945C176B
:101FC00080FD5DC1F70112820E9456170E94DF1545
:101FD000C7010E9460110E945617DF91CF911F9197
:101FE0000F91FF90EF90DF90CF90BF900C94001670
:101FF000812F0E948017D4CF2C2F2F70B22EC07F3C
:10200000C03219F0B29480EFB822DD2339F0D1301C
:1020100019F1002361F1112321F1ACCF002381F0EC
:10202000111106C00E948D178B290E945D0FBACF37
:102030001130C1F70E948D178B290E949317B2CFE0
:10204000111106C00E949C178B2D0E94640FAACF0D
:10205000113009F4A7CFF6CF002329F0163008F08D
:10206000A1CF8B2DE2CF153008F09CCFEDCF1123FF
:1020700059F3D93349F43FEF87EE93E03150804074
:102080009040E1F700C000008D2F0E94220F8ACF00
:102090008C2F837009F041C0011184CF4D2F4295E0
:1020A00046954770440F440F0D2F0F7010E030E03D
:1020B00020E0042E04C0000F111F221F331F0A94BA
:1020C000D2F760E070E0CB01D4FF0FC06FE070E0AA
:1020D00080E090E004C0660F771F881F991F4A9523
:1020E000D2F76095709580959095C695C695C3700A
:1020F000602B712B822B932BC23049F058F4C130E6
:1021000019F00E9491154ECF0E947F154BCF0E946F
:10211000A31548CF0E947D1545CF8695002311F069
:102120008C2F8170882309F43DCF4D2F4295469521
:102130004770440F440F0D2F0F7010E030E020E087
:10214000042E04C0000F111F221F331F0A94D2F760
:1021500060E070E0CB01D4FF0FC06FE070E080E082
:1021600090E004C0660F771F881F991F4A95D2F729
:102170006095709580959095C695C695C370602BB7
:10218000712B822B932BC23049F058F4C13019F0D7
:102190000E94561607CF0E94441604CF0E9468166C
:1021A00001CF0E94B915FECECF70002329F08C2FED
:1021B0000E94DF158D2F39CF8D2F0E94640F8C2F39
:1021C0000E940016EFCED23F89F160F4D03FC9F0F3
:1021D000D13F29F1002309F442C01111CBCE8C2F3D
:1021E0008F7121C0D33F39F1D43FA1F7002369F1AA
:1021F000CF718C2F0E94DF1563E08C2F0E94DC17BB
:10220000D1CE002341F0153008F0CCCE8C2F8F7149
:102210000E942316C7CE163008F0C4CEF7CF8C2FFD
:102220008F71002369F20E94DF15BCCE8C2F8F7155
:102230000023C9F3C5CF002329F08C2F8F710E9492
:10224000CA15B0CE0E94C515ADCE81E00E94F1172F
:10225000123008F4A7CE82E00E94F117A3CE11231A
:1022600059F0D93309F010CFEFEFF7EE23E0E1504A
:10227000F0402040E1F706CF8C2F8F71A1CFDF9186
:10228000CF911F910F91FF90EF90DF90CF90BF9073
:1022900008950F931F93CF93DF93EC0168817981A9
:1022A0008A810E941E178C010E947A160E947C155A
:1022B000B801CE01DF91CF911F910F910C946B0F5C
:1022C000CF93DF93EC018B819C81892B29F088814E
:1022D000998189238F3F59F4DF91CF910895CE01E1
:1022E0000E944911CE01DF91CF910C946802CE017A
:1022F0000E94BF038111F3CF0E946017882361F30E
:102300008A81882349F382E0DF91CF910C94F11701
:102310000E9487170E948A170C94A6170E945017D4
:102320000C9488110E9477170C948E11E92FE29576
:10233000EF70E250EE3070F4F0E0E456FE4D0C9495
:102340002C21803F19F020F4883E20F481E008958C
:10235000843FE1F380E00895883EC0F3813FD1F7E8
:10236000F5CF93FB882780F908950E9414170C94E9
:102370009611CF93DF9300D000D00F92CDB7DEB788
:102380000F900F900F900F900F90DF91CF910895C5
:10239000CF93DF9300D000D000D0CDB7DEB7269624
:1023A0000FB6F894DEBF0FBECDBFDF91CF91089579
:1023B0001F93CF93DF93C091440116E080914501B4
:1023C0008C1304C0DF91CF911F910895D0E01C9F22
:1023D000F0011D9FF00D1124EA5BFE4F40815181F9
:1023E00062817381848195810E94C8112196C77092
:1023F000E5CF40917601509177016091780170911D
:10240000790180917A0190917B010C94C8112091FF
:1024100044019091450156E0291302C080E00895DF
:1024200030E0529FF001539FF00D1124EA5BFE4F04
:102430007181761306C07081781303C072817413A2
:1024400004C02F5F3F4F2770E7CF81E00895DF92F0
:10245000EF92FF920F931F93CF93DF9380917B01B5
:10246000807F61F480917801882341F0C09144011C
:1024700086E0D82E809145018C1308C0DF91CF9162
:102480001F910F91FF90EF90DF90089520917901B7
:1024900030917A01D0E02115310541F0809176012B
:1024A00090917701482F49234F3F19F42196C77027
:1024B000E1CFDC9E8001DD9E100D1124F801EA5B66
:1024C000FE4F51815913F2CF40814813EFCF8281E3
:1024D0008111ECCFE380F480E21AF30A20E06091EE
:1024E00078017091790180917A010E942C0266E74F
:1024F00071E00E94EB01E816F906C0F680917B01BD
:102500008F70806180937B01F801E55BFE4F8081D5
:102510008F708061808386E791E00E946011DF9177
:10252000CF911F910F91FF90EF90DF900C94D811F5
:102530006F927F928F929F92AF92BF92CF92DF92D3
:10254000EF92FF920F931F93CF93DF93CDB7DEB738
:1025500061970FB6F894DEBF0FBECDBF8C0185E04A
:10256000F801DE011D9601900D928A95E1F7D801E0
:102570007C901196EC9011971296FC9086E7882E2D
:1025800081E0982E8091790190917A01009749F02D
:102590004091760150917701242F25232F3F09F098
:1025A0009DC1F11009C1C8010E94601175C0CD28FC
:1025B00029F08E2D87218F3F09F017C180E0B82FB9
:1025C000B170CB2E80FF29C04F2D6E2D872D0E941C
:1025D0000712D82E811121C07D86EE868D859E85BD
:1025E0000E941417292F22952F70223050F024308A
:1025F00078F49F7051F0F8019581907F31F46D2C43
:1026000010C19F7011F08823D1F3805E8830B8F339
:10261000C8010E946011DC2CF2CFFF2009F401C137
:1026200080917B01816080937B01612CFAC0892BB2
:1026300049F08091760190917701282F29232F3F2F
:1026400009F005C17D86EE868D859E850E94B511B7
:10265000882309F4A8CFFF2009F4A5CF80917B013E
:10266000803270F0209176013091770138872F8386
:102670001986DB86CA868C87CE0107960E94601178
:1026800086E0F801A6E7B1E001900D928A95E1F7A6
:102690000E9427120E94F91166246394C2C021117E
:1026A00013C07C2DD98AC88A472D5E2D6F2D89894C
:1026B0000E94B91186E791E00E94601186E0F40162
:1026C00011928A95E9F76CC18091790190917A0114
:1026D000892B49F08091760190917701282F292349
:1026E0002F3F09F0CDC07D86EE868D859E850E94A8
:1026F000B511882309F457CFFF2009F454CF8091F6
:102700007B01803208F4BCCF2091760130917701B3
:102710003A8329831B82DD82CC828E83CE0101968F
:10272000ADCF20E060E07091790180917A010E9444
:102730002C0266E771E00E94EB01A816B90668F565
:102740006F2CFF2009F42FCF8091790190917A01AD
:10275000892B49F08091760190917701282F2923C8
:102760002F3F09F0A3C07D86EE868D859E850E9451
:10277000B511811185CF80917B01816080937B01B0
:10278000C8010E9460114DC086E0F801A6E7B1E0E3
:1027900001900D928A95E1F744C07C2DD98AC88AB0
:1027A000472D5E2D6F2D89890E94B91186E0D401D5
:1027B0001D928A95E9F761C07D86EE868D859E859E
:1027C0000E94B511682E882309F4EDCE86E0F80149
:1027D000A6E7B1E001900D928A95E1F786E791E0D6
:1027E0000E94F20E0E94271248C081E08F25E7CE9A
:1027F00081E08F25C0C09E11A1C087119FC0F1103C
:102800009DC080917B018F70806180937B010E94CD
:10281000F91186E791E00E94601180917B01F80137
:102820008583862D61960FB6F894DEBF0FBECDBFAF
:10283000DF91CF911F910F91FF90EF90DF90CF909C
:10284000BF90AF909F908F907F906F9008959E1152
:10285000F9CE8711F7CEF110F5CE80917B01D8012A
:1028600015968C93C8010E94601186E0F801A6E7D6
:10287000B1E001900D928A95E1F70E94F911D1CF54
:102880009E1131CF87112FCFF1102DCF80917B0179
:10289000D80115968C93C8010E946011E6E7F1E01B
:1028A00086E0DF011D928A95E9F7BBCF9E115BCFD1
:1028B000871159CF90917B0190FD66CF907F09F4ED
:1028C00063CF80917B01F8018583903F59F2982F67
:1028D000907F905F8F70892B8583C4CFF801C38070
:1028E000D480609078015601A81AB90A662009F4CC
:1028F00018CF20E0662D7091790180917A010E94B5
:102900002C0266E771E00E94EB0120917B01207FA1
:10291000A816B90608F0C3CE8091790190917A018A
:10292000211185CE6F2C892B49F0809176019091F1
:102930007701282F29232F3F09F05DCF20E0409118
:1029400076015091770160917801709179018091C1
:102950007A010E942C02B8010E94EB01843F914051
:1029600008F425CEC114D10429F08E2D87218F3F84
:1029700009F03ECF80E080FF1ACE4F2D6E2D872DBF
:102980000E940712882309F412CE86E791E00E9484
:10299000601186E0E6E7F1E0DF011D928A95E9F734
:1029A0000E94F91142CE1F93CF93DF93CDB7DEB7CC
:1029B0002C970FB6F894DEBF0FBECDBF4F8358875C
:1029C00069877A878B879C87CE0107960E94981229
:1029D000882369F08A859B85892B39F04F8158853A
:1029E000842F85238F3F09F071C016E05FC086E019
:1029F000FE013796DE01119601900D928A95E1F75E
:102A00008A859B85892B89F38F81988589238F3FC0
:102A100061F32091450130E0C90101968770992743
:102A2000409144014817190671F40E9492111092C6
:102A300045011092440186E0E6E7F1E0DF011D92D6
:102A40008A95E9F7D2CF96E0929FD001939FB00D7F
:102A50001124AA5BBE4FFE01319601900D929A950A
:102A6000E1F7809345010E94D811BFCF819FC0013B
:102A700011248A5B9E4F0E9498128823E9F0E0910E
:102A800044011E9FF0011124EA5BFE4F40815181F9
:102A900062817381848195810E94C8118091440173
:102AA00090E00196877099278093440180914401BA
:102AB000909145018913DACF2C960FB6F894DEBFBA
:102AC0000FBECDBFDF91CF911F91089569857A85A3
:102AD0008B859C850E94C81188CF08950C946D1534
:102AE0000E946E1560939E0170939F018093A001D8
:102AF0009093A1010C94881108950C9470150F9374
:102B00001F9300919E0110919F012091A00130918F
:102B1000A101602B712B822B932B1F910F910C9491
:102B200070150F931F9300919E0110919F012091AA
:102B3000A0013091A10160237123822393231F916F
:102B40000F910C9470150F931F9300919E0110919B
:102B50009F012091A0013091A10160277127822758
:102B600093271F910F910C9470150C946D150C9474
:102B7000B5150E94B71560939A0170939B018093DD
:102B80009C0190939D010C94881160E070E0CB0152
:102B90000C94B9150F931F9341E050E060E070E092
:102BA0008A019B0104C0000F111F221F331F8A9549
:102BB000D2F7C901B8011F910F910C94B9150F9369
:102BC0001F9341E050E060E070E004C0440F551FE7
:102BD000661F771F8A95D2F780919A0190919B0189
:102BE000A0919C01B0919D018A019B01082B192B9A
:102BF0002A2B3B2BC901B8011F910F910C94B915D9
:102C00000F931F9341E050E060E070E004C0440F78
:102C1000551F661F771F8A95D2F7CB01BA016095C1
:102C200070958095909500919A0110919B0120914B
:102C30009C0130919D0160237123822393231F9176
:102C40000F910C94B9150F931F9341E050E060E091
:102C500070E004C0440F551F661F771F8A95D2F796
:102C600080919A0190919B01A0919C01B0919D014E
:102C70008A019B01082719272A273B27C901B80188
:102C80001F910F910C94B9150F931F9300919A0106
:102C900010919B0120919C0130919D01602B712B23
:102CA000822B932B1F910F910C94B9150F931F93A7
:102CB00000919A0110919B0120919C0130919D01FE
:102CC00060237123822393231F910F910C94B915D4
:102CD0000F931F9300919A0110919B0120919C01E9
:102CE00030919D0160277127822793271F910F91B3
:102CF0000C94B9150895E92FEE0FE90FEE0F8E0F22
:102D0000982F977041E001C0440F9A95EAF7869595
:102D10008695869595E0899FF0011124E458FE4F31
:102D200030E020E070E05191DF011197CB01022EDD
:102D300002C0969587950A94E2F781708195852760
:102D4000842385278C932F5F3F4F2530310559F71A
:102D50000895E92FEE0FE90FEE0F8E0F982F977061
:102D600086958695869525E0829FF0011124E4588A
:102D7000FE4F50E040E080E0219130E0092E02C09B
:102D8000369527950A94E2F721703327042E01C067
:102D9000220F0A94EAF7822B4F5F5F4F45305105AF
:102DA00059F70895BF92CF92DF92EF92FF920F935F
:102DB0001F93CF93DF938C01C0909A01D0909B0119
:102DC000E0909C01F0909D0180919E0190919F0167
:102DD000A091A001B091A101C82AD92AEA2AFB2A10
:102DE000CFE1D0E0BC2ED701C6010C2E04C0B695B1
:102DF000A795979587950A94D2F780FD0EC02197E5
:102E000088F7B12C8B2DDF91CF911F910F91FF90FF
:102E1000EF90DF90CF90BF900895B8018C2F0E9463
:102E20001004019761F3EECFCF93DF93EC010E9482
:102E3000D216BE01DF91CF910C9410041F93CF9353
:102E4000DF93EB0190914301992331F0CB01DF91A6
:102E5000CF911F910C941417882379F0CB010E9415
:102E6000D216182F682FCE010E947B16BE01812F2B
:102E7000DF91CF911F910C941004CB010E94A916F1
:102E8000182FF4CF682F8091090190910A010C94BA
:102E90000719682F8091090190910A010C94091972
:102EA0008091090190910A010C940B198091A20163
:102EB00085958595859508958091A20187700895DF
:102EC0009091A201977081E009F480E008958091CB
:102ED000AE0108959091AE01892B8093AE010895C3
:102EE00080959091AE0198239093AE010895109231
:102EF000AE0108959091AD01892B8093AD010895A5
:102F000080959091AD0198239093AD010895109212
:102F1000AD0108951092AC0108958091A301089528
:102F200008950C9490179091A301981721F0809325
:102F3000A3010C94911708958091A301882329F08F
:102F40001092A30180E00C9491170895E09109017B
:102F5000F0910A018091AE018083E0910901F09126
:102F60000A0180819091AD01892B8083E091090154
:102F7000F0910A0180819091AC01892B808390911E
:102F8000A301992381F0E0910901F0910A01808168
:102F9000892B80838091090190910A010E94BF18BA
:102FA00081110E949C178091090190910A010C9453
:102FB000D60D08950C94D91798E0899F900111249B
:102FC000622B6093A2010E94DF158091A20185957A
:102FD000859585950C94DA171092A20180E00C94E7
:102FE000DA179091A201809589238093A201282F5E
:102FF000277071F4282F082E000C330B921713063C
:1030000039F08595859585950E9400160C94EC17EE
:1030100008956FEF7FEF90E080E00C94652190E0E1
:1030200080E00E94412121E08C3E9E4F09F020E08B
:10303000822F089582E090E00C94392183E090E0A3
:103040000C943921682F83E090E00C944721CF93B2
:1030500084E090E00E943921C82F81E290E00E9434
:103060003921982F8C2FCF910895CF93C92F682F96
:1030700084E090E00E9447216C2F81E290E0CF91A4
:103080000C944721AB01BC018FE090E00C945921D6
:10309000AB01BC0183E190E00C94592160E070E049
:1030A000CB010C94481860E070E0CB010E944218FC
:1030B0000C944E186CEE7EEF90E080E00E9465214B
:1030C00060E082E090E00E94472160E083E090E0D1
:1030D0000E94472110929E0110929F011092A00120
:1030E0001092A10160E084E090E00E94472160E03E
:1030F00081E290E00E94472160E085E090E00E943C
:10310000472160E086E090E00E9447216FEF87E072
:1031100090E00E94472140E050E0BA0188E090E052
:103120000E94592160E08DE090E00E94472140E03C
:1031300050E0BA0188E190E00E94592160E087E107
:1031400090E00E94472140E050E0BA018CE190E01D
:103150000E94592160E080E290E00E94472140E017
:1031600050E0BA0188E190E00E9459210C94531874
:103170000C945A18682F8EE090E00C9447219C0123
:103180002E5F3F4FAC01485F5F4F80E0241735074B
:1031900009F40895F90191919F019923B9F38F5F83
:1031A000F5CF662349F0FC01329608962191261747
:1031B00029F0E817F907D1F780E0089581E0089534
:1031C0009C01FC0132969FEF80E04191461751F03F
:1031D0009F3F19F4411101C0982F8F5F8630A9F7E6
:1031E0009F3F09F40895290F311D97FD3A95F90184
:1031F00062830895FC01329608962191261303C03C
:10320000DF0111971C92E817F907B9F708950C949C
:10321000E0180C94FA18029626E0FC0111922A9507
:10322000E9F70895089508950C9413190E9414194C
:103230008091D701843049F11092B00188E190E08B
:1032400020E40FB6F894A895809360000FBE2093F9
:10325000600080E00E9408040E94141983B7817FF7
:10326000846083BF83B7816083BF7894889583B778
:103270008E7F83BF0FB6F894A89580916000886117
:1032800080936000109260000FBE08950895CF9360
:103290000E9412190E944F060E944619C0E08C2F0E
:1032A0000E94C205811105C0CF5FC830C1F7CF9120
:1032B000089581E0FCCF08950C945B190E9492114F
:1032C0000E94CA0D0E9408040C945C191F921FB63C
:1032D0001F9211248F939F93AF93BF938091B0015E
:1032E000811113C08091CD019091CE01A091CF01A9
:1032F000B091D0014196A11DB11D8093CD01909355
:10330000CE01A093CF01B093D001BF91AF919F9117
:103310008F911F901FBE1F90189582E084BD93E08F
:1033200095BD9AEF97BD80936E0008952FB7F894DE
:103330008091CD019091CE01A091CF01B091D001AB
:103340002FBF08952FB7F8946091CD017091CE01F1
:103350008091CF019091D0012FBF08959C014FB76C
:10336000F8948091CD019091CE01A091CF01B091C0
:10337000D0014FBF821B930B089578941F921FB604
:103380001F9211248F939F93AF93BF938091CD0190
:103390009091CE01A091CF01B091D0010196A11DD5
:1033A000B11D8093CD019093CE01A093CF01B09336
:1033B000D001BF91AF919F918F911F901FBE1F9021
:1033C000189587E797E7909301088093000888E1B4
:1033D0009AE00FB6F894A895809360000FBE909382
:1033E0006000FFCF0C9492070E944F068FE39CE988
:1033F0000197F1F700C000000E944F0680E00E9494
:10340000C20580FF04C00E94F2190C94E1190895CE
:103410000E940F18811102C00E94B8180E941A1849
:103420008093AF010E9427189093D2018093D1011D
:103430000E941E18682F70E090E080E00E947D15C9
:1034400060919A0170919B0180919C0190919D01E6
:103450000C94B7158091B901089508950895CF93FC
:10346000DF93EC0181E08093E9008FEF9091E80019
:10347000815095FD06C095ED9A95F1F700008111F8
:10348000F5CF8091E80085FF14C050E040E068E08F
:1034900070E0CE010E944C1C8091E8008E778093F2
:1034A000E80088E0FE01A1EBB1E001900D928A9561
:1034B000E1F7DF91CF9108950895CF93FC01603239
:1034C00021F58091D701843001F5C091E900CF70DA
:1034D0002091EC00922F917020FD90E8C92B82E0A2
:1034E0008093E9008091E80080FF0CC050E040E04C
:1034F00060E270E0CF010E944C1C8091E8008E7762
:103500008093E800CF70C093E900CF910895809137
:10351000D601811109C00E942B1E0E94881E809135
:10352000E20084608093E20008951092D60108952D
:10353000089508950C945E1942E061EC81E00E94C8
:10354000A71D42E261EC82E00E94A71D42E260EC0E
:1035500083E00C94A71D8091D901833009F45FC0EA
:1035600030F48130C1F1823009F49BC008958A3073
:1035700009F487C08B3009F46DC0893009F04EC062
:103580008091D801813209F049C08091DC0190918D
:10359000DD01892B09F042C08091E800877F80938C
:1035A000E8008091E80082FF35C09091F30080919F
:1035B000F200029729F48091F1008B7F813021F491
:1035C0008091F1008093B9018091E8008B7780931E
:1035D000E8000C94DB1D8091D801813AF9F48091C8
:1035E000E800877F8093E8008091DC019091DD0105
:1035F000892B61F468E081EB91E070E00E94EA1CA5
:103600008091E8008B778093E800089560E090E077
:1036100080E0F3CF8091D7018111C3CF08958091CD
:10362000D801813AD9F78091DC019091DD01892B95
:10363000A9F78091E800877F8093E8008091E800F7
:1036400080FFFCCF809115018093F1008091E8000C
:103650008E77BDCF8091D801813201F78091DC0156
:103660009091DD01892BD1F68091E800877F8093CE
:10367000E8000E94DB1D8091DA01809315010C9413
:1036800092118091D801813249F68091E800877FBC
:103690008093E8000E94DB1D8091DB018093BA01DA
:1036A00008958091D801813A09F0B8CF8091E8005F
:1036B000877F8093E8008091E80080FFFCCF8091B5
:1036C000BA01C2CFCDB7DEB7A0970FB6F894DEBF70
:1036D0000FBECDBF84B7877F84BF0FB6F894A8957F
:1036E00080916000886180936000109260000FBE3E
:1036F00080E890E00FB6F8948093610090936100A9
:103700000FBE0E941B0E0E942B1E0E94881E8091DD
:10371000E20084608093E20078940E9411210E946C
:10372000250E8BE091E00E94C50D13E08091D7013A
:10373000853059F00E942F0E8091D701843091F08E
:103740000E94230E0E94240EF1CF0E941619809130
:10375000D501882359F30E944719882339F30E9421
:10376000361CE4CF1093E9008091E80082FFE8CF97
:103770008091E80090E085FF09C050E040E060E201
:1037800070E0CE0101960E949B1C91E08091E800C0
:103790008B778093E800992399F260E2CE0101963D
:1037A0000E94F407CDCF0C94D51BE92FFF27E330FF
:1037B000F105E9F060F4E130F10509F448C0329711
:1037C00009F44AC0F0E0E0E090E080E025C0E1329A
:1037D000F10571F1E232F105A9F76115710509F4FE
:1037E00040C082EE92E061307105B1F0EBCF9927D5
:1037F00081309105B1F0009749F0029719F7ECE696
:10380000F2E0E491F0E08CE692E006C0EAE8F2E053
:10381000E491F0E08AE892E0DA018D939C93CF0185
:103820000895ECE7F2E0E491F0E08CE792E0F4CF69
:10383000E9E0F0E080EA92E06115710569F3E9E002
:10384000F0E089EB92E06130710531F3BBCFE2E14A
:10385000F0E080ED92E0E0CFE2E4F0E08EE892E08C
:10386000DBCFE0E4F0E084E093E0D6CF80E189BDF7
:1038700082E189BD09B400FEFDCF8091D8008F7D23
:103880008093D8008091E00082608093E000809176
:10389000E00081FDFCCF0895AF92BF92CF92DF92FE
:1038A000FF920F931F93CF93DF936C01EB018A017B
:1038B0000E94FA1DF82E811123C00115110539F05F
:1038C000F80180819181C81BD90BC80ED91EB12C7B
:1038D000A12C2097A9F08091E80085FD22C080915D
:1038E000E8008E778093E80001151105A1F0F8013A
:1038F00080819181A80EB91EB182A08285E0F82E48
:103900008F2DDF91CF911F910F91FF90DF90CF907E
:10391000BF90AF9008950E94FA1D8823D1F2F82E2F
:10392000EFCFF60181916F018093F1002197FFEFB6
:10393000AF1ABF0ACECFAF92BF92CF92DF92FF9263
:103940000F931F93CF93DF936C01EB018A010E94C9
:10395000FA1DF82E811123C00115110539F0F80167
:1039600080819181C81BD90BC80ED91EB12CA12C06
:103970002097A9F08091E80085FD22C08091E800A1
:103980008B778093E80001151105A1F0F801808183
:103990009181A80EB91EB182A08285E0F82E8F2DEC
:1039A000DF91CF911F910F91FF90DF90CF90BF904B
:1039B000AF9008950E94FA1D8823D1F2F82EEFCF20
:1039C0008091F100F60181936F012197FFEFAF1A0B
:1039D000BF0ACECFFC018091DE019091DF018617F6
:1039E0009707A0F06115710529F49091E8009E7782
:1039F0009093E80090E06115710551F4911108C0B1
:103A00008091E80082FF34C080E00895BC01F2CFCD
:103A10008091D7018823C1F18530C1F18091E80000
:103A200083FD30C08091E80082FDEACF8091E800FC
:103A300080FFE1CF8091F3002091F200382F6115D3
:103A4000710519F02830310558F091E02830310522
:103A500009F090E02091E8002E772093E800CBCF8A
:103A600081918093F100615071092F5F3F4FE7CF43
:103A70008091D701882341F0853041F08091E800A2
:103A800083FFBECF81E0089582E0089583E008952A
:103A9000FC018091DE019091DF0186179707A0F06D
:103AA0006115710529F48091E8008E778093E80014
:103AB00090E06115710551F4911108C08091E80002
:103AC00082FF35C080E00895BC01F2CF8091D7011C
:103AD0008823C9F18530C9F18091E80083FD31C0A8
:103AE0008091E80082FDEACF8091E80080FFE1CF7D
:103AF0008091F3002091F200382F6115710519F0C3
:103B00002830310558F091E02830310509F090E077
:103B10008091E8008E778093E800CBCF84918093EA
:103B2000F1003196615071092F5F3F4FE6CF8091D0
:103B3000D701882341F0853041F08091E80083FF70
:103B4000BDCF81E0089582E0089583E00895982F25
:103B5000973028F08F708093E90081E0089590936A
:103B6000E900242F762F50E0981731F07091EC0087
:103B70002091ED005091F00021FD02C09F5FE8CF41
:103B80003091EB003E7F3093EB003091ED003D7FB4
:103B90003093ED003091EB0031603093EB00709387
:103BA000EC002093ED005093F0002091EE0027FDF3
:103BB000E5CF80E008958091D80187FF13C0809100
:103BC000E80082FF06C08091E8008B778093E800D0
:103BD00004C08091D7018111F2CF08958091D7015F
:103BE0008823D9F38091E80080FFF8CF8091E80026
:103BF0008E77ECCF2091E4003091E50095E6A901A5
:103C00002091EC00822F817020FF06C08091E80097
:103C100080FF06C080E008952091E80022FD1AC0D0
:103C20008091D701882389F0853089F08091EB005D
:103C300085FD0FC02091E4003091E5004217530745
:103C4000F9F29150E1F684E0089582E0089583E06E
:103C5000089581E008950E94991E0E94A11EE0EE41
:103C6000F0E0808181608083E8EDF0E080818F77F3
:103C7000808319BCA7EDB0E08C918E7F8C938081FE
:103C80008F7E80831092D60108950F931F93CF9358
:103C9000DF930E94991E0E94A11EC8EDD0E088818A
:103CA0008F77888388818068888388818F7D8883E7
:103CB00019BC1092D7011092D3011092D501109225
:103CC000D40100EE10E0F80180818B7F8083888131
:103CD0008160888342E060E080E00E94A71DE1EE01
:103CE000F0E080818E7F8083E2EEF0E08081816071
:103CF0008083808188608083F80180818E7F8083CB
:103D0000888180618883DF91CF911F910F91089501
:103D1000E8EDF0E080818F7E8083E7EDF0E0808148
:103D20008160808384E082BF81E08093D6010C941F
:103D3000451EE8EDF0E080818E7F80831092E200E6
:103D400008951092DA001092E10008951F920F92E8
:103D50000FB60F9211242F933F934F935F936F935E
:103D60007F938F939F93AF93BF93EF93FF93809134
:103D7000E10082FF0BC08091E20082FF07C08091CA
:103D8000E1008B7F8093E1000E9410218091DA0096
:103D900080FF19C08091D80080FF15C08091DA00A3
:103DA0008E7F8093DA008091D90080FF96C080E1F9
:103DB00089BD82E189BD09B400FEFDCF81E0809319
:103DC000D7010E94871A8091E10080FF19C080917D
:103DD000E20080FF15C08091E2008E7F8093E200B8
:103DE0008091E20080618093E2008091D80080623F
:103DF0008093D80019BC85E08093D7010E94991A5E
:103E00008091E10084FF2BC08091E20084FF27C0F5
:103E100080E189BD82E189BD89B5982F917080FFCD
:103E2000FBCF8091D8008F7D8093D8008091E100F6
:103E30008F7E8093E1008091E2008F7E8093E2008C
:103E40008091E20081608093E2008091D301882319
:103E500009F449C084E08093D7010E949A1A8091A6
:103E6000E10083FF29C08091E20083FF25C080919B
:103E7000E100877F8093E10082E08093D701109278
:103E8000D3018091E1008E7F8093E1008091E20078
:103E90008E7F8093E2008091E20080618093E20057
:103EA00042E060E080E00E94A71D8091F000886001
:103EB0008093F0000E94981AFF91EF91BF91AF910B
:103EC0009F918F917F916F915F914F913F912F9132
:103ED0000F900FBE0F901F90189519BC1092D7012C
:103EE0000E94951A70CF8091E30087FD93E0909334
:103EF000D701B3CF1F920F920FB60F9211242F93B9
:103F00003F934F935F936F937F938F939F93AF9361
:103F1000BF93CF93DF93EF93FF93D091E900DF70CE
:103F20008091EC00C82FC17080FDC0E81092E900BC
:103F30008091F000877F8093F00078940E94BE1FEC
:103F40001092E9008091F00088608093F000CD2B02
:103F5000CF70C093E900FF91EF91DF91CF91BF91B6
:103F6000AF919F918F917F916F915F914F913F9111
:103F70002F910F900FBE0F901F9018951F93CF9306
:103F8000DF93CDB7DEB7AA970FB6F894DEBF0FBEAA
:103F9000CDBF88ED91E02091F100FC012193CF018C
:103FA000F1E0803E9F07B9F70E94AB1A8091E800CC
:103FB00083FF1EC18091D8019091D9019A3008F0F9
:103FC00017C1E92FF0E0E655FE4D0C942C21803806
:103FD00099F0823809F00CC18091DC018F70873034
:103FE00008F006C18093E9008091EB0085FB8827EB
:103FF00080F91092E90006C08091D4019091D5011A
:10400000911182609091E800977F9093E8008093EF
:10401000F1001092F1008091E8008E77E5C08823CE
:1040200009F4D3C0823009F0E3C08091DA01811134
:10403000D6C08091DC018F702FEF280F263008F05A
:10404000D7C08093E9002091EB0020FFC8C09330D7
:1040500031F48091EB0080628093EB00C0C09091BE
:10406000EB0090619093EB0021E030E001C0220F63
:104070008A95EAF72093EA001092EA008091EB001B
:104080008860EACF8111B4C01091DA011F77809166
:10409000E3008078812B8093E3008091E800877FA4
:1040A0008093E8000E94DB1D8091E80080FFFCCF38
:1040B0008091E30080688093E30082E0111183E047
:1040C0008093D70195C08058823008F091C08091CC
:1040D000DA019091DB018C3D23E09207A1F583E0AA
:1040E0008A838AE289834FB7F894DE01139620E031
:1040F0003EE051E2E32FF0E050935700E49120FFBF
:1041000003C0E295EF703F5FEF708E2F90E0EA30D2
:10411000C0F0C7968D939D932F5F243159F74FBF01
:104120008091E800877F8093E8006AE270E0CE012A
:1041300001960E94EA1C8091E8008B778093E8004A
:1041400057C0C096E7CF6091DC017091DD01AE01F0
:104150004F5F5F4F0E94D31BBC01892B09F448C0FD
:104160009091E800977F9093E80089819A810E945E
:10417000481DE1CF8038E1F58091E800877F80938A
:10418000E8008091D3018093F10045CF811130C0C8
:104190009091DA01923060F58091E800877F8093FA
:1041A000E8009093D3010E94DB1D8091D301882306
:1041B00011F084E005C08091E30087FDFACF81E033
:1041C0008093D7010E949C1A13C08091DA0181303C
:1041D00079F481E0933009F080E08093D50110926A
:1041E000E9008091E800877F8093E8000E94DB1D52
:1041F0008091E80083FF0AC08091E800877F809368
:10420000E8008091EB0080628093EB00AA960FB6E5
:10421000F894DEBF0FBECDBFDF91CF911F910895FF
:104220000895CF938091D7018823A1F0C091E90030
:10423000CF709091EC00892F817090FD80E8C82BA1
:104240001092E9008091E80083FD0E94BE1FCF70AC
:10425000C093E900CF910895EE0FFF1F0590F491F0
:10426000E02D0994692796276927782787277827DB
:104270000895F999FECF92BD81BDF89A992780B52E
:104280000895A8E1B0E042E050E00C946D21262FA3
:10429000F999FECF92BD81BDF89A019700B402163C
:1042A00039F01FBA20BD0FB6F894FA9AF99A0FBEEA
:1042B00008950396272F0E9448210E944721252F09
:1042C0000E944821242F0C9448210196272F0E94F8
:1042D00048210C944721DC01CB01FC01F999FECF68
:1042E00006C0F2BDE1BDF89A319600B40D9241507E
:1042F0005040B8F70895F894FFCF060813083A081D
:10430000460851085C085F085F085F08A808AB080A
:10431000620866086E087B0888088B088E089B0870
:10432000A50FA50FFC0FFC0FD20FD20FD20FD20F8B
:104330004810D410E310E310A111A111AA11AA1181
:10434000AC11AA11AA11AA11A111A111B111AA119E
:10435000AA11B111E71F0F20F8200F20F8204220EA
:084360006320F820BA20C620FA
:10436800012901002A01042A01A4012A1A2F1A2D61
:104378001A2E1A5C1A01F4F5F6F73133946697C6CB
:044388000000000031
:00000001FF
